:0400000006EF1AF0FD
:1000080000C015F0E1CF16F0E2CF17F09EAA4BD052
:100018009DAA49D0AFCF1AF0ACA202D0AC98AC8858
:10002800ACA402D0AFCF1AF01A500D0A14E1010E99
:100038002D6E000E2E6EBC0E00019C25E16E000E8A
:100048009D21E26EE66A9CC018F09DC019F09C6B79
:100058009D6B1A6A0FD00001BC0E9C25E16E000E44
:100068009D21E26E1AC0E6FF9CC018F09DC019F0F1
:100078009C4B9D2B000E9D5D02E1800E9C5D13E361
:10008800020E2D6E000E2E6E9D9ABC0E9C25E16E02
:10009800000E9D21E26EE66A9CC018F09DC019F022
:1000A8009C6B9D6B1A6AA4AA54D0A3AA52D09CA296
:1000B80002D09C989C889CA404D0AACFD2F20201BA
:1000C800D26B0201AACFD2F2D2510A0A14E1010E70
:1000D8002B6E000E2C6E400E00016925E16E010E9C
:1000E8006A21E26ED2C2E6FF69C063F06AC064F0BA
:1000F8000201D26B0FD0400E00016925E16E010E9E
:100108006A21E26ED2C2E6FF69C063F06AC064F099
:10011800694B6A2B0001010E6A5D02E1000E695D00
:1001280018E3020E2B6E000E2C6EA39A010E695F67
:10013800000E6A5B400E6925E16E010E6A21E26ECF
:10014800E66A69C063F06AC064F0696B6A6B0201B1
:10015800D26BF2AA1AD0F2A418D00301B84BB92B6B
:10016800000E006EB951005C02E1B851090808E2BE
:10017800010EAA6F000EAB6FF29AB86BB96BD59EE1
:10018800480ED76EE50ED66EF2949DA01BD09EA0A9
:1001980019D00301B64BB72B000E006EB751005CA7
:1001A80002E1B651640804E2240EAE6EB66BB76B7A
:1001B800010EB46F000EB56FCD906D0ECF6E840E2C
:1001C800CE6E9E9015C000F016C0E1FF17C0E2FF8A
:0201D800110014
:1001DA000B820BAEF7EF00F0036802680168006853
:0801EA000A360232FF0E12007A
:0E01F200026A016A006A086A036A000E1200BF
:100200000B840BAE0BEF01F0010E036E026A016A64
:0A021000006A0A360232FF0E1200E7
:08021A000AAE029E000E120064
:10022200C7B409D01F0EC514016E0150000A03E1C4
:0A023200010E006E01D0006A1200F8
:10023C000CB060EF01F00CA206EF02F00E6A000E9B
:10024C00026477EF01F0F00E0214D8A442EF01F033
:10025C00023A01380F0B02260138F00B016E003800
:10026C000F0B01260038F00B006E08380F0B002620
:10027C000838F00B086E0E84D89002BE5BEF01F0CC
:10028C0008360036013602360E2A02BE5BEF01F04C
:10029C0008360036013602360E2A02BE5BEF01F03C
:1002AC0008360036013602360E2A0E500364FCEF77
:1002BC0001F0035E0BBC08AE01EF02F0D880800E9B
:1002CC0008640030000E002201220222D8A001EFA7
:1002DC0002F0023201320032034A06EF02F001EF63
:1002EC0002F001C002F000C001F008C000F0086A82
:1002FC00000E0E860264AEEF01F0F00E0214D8A4CC
:10030C0096EF01F0023A01380F0B02260138F00B80
:10031C00016E00380F0B01260038F00B006E0E84B6
:10032C00D89002BE5BEF01F00036013602360E2A81
:10033C0002BE5BEF01F00036013602360E2A02BE19
:10034C005BEF01F00036013602360E2A5BEF01F04E
:10035C0001C002F000C001F0006A000E0E960E887B
:10036C000264DBEF01F0F00E0214D8A4C6EF01F02A
:10037C00023A01380F0B02260138F00B016E0E8485
:10038C00D89002BE5BEF01F0013602360E2A02BE97
:10039C005BEF01F0013602360E2A02BE5BEF01F074
:1003AC00013602360E2A5BEF01F001C002F0016A41
:1003BC00000E0E8602640BEF02F0F00E0214D8A4AD
:1003CC00EAEF01F0023A0E84D89002BE5BEF01F026
:1003DC0002360E2A02BE5BEF01F002360E2A02BE76
:1003EC005BEF01F002360E2A5BEF01F0010E0C6E92
:1003FC0001DF0EEF02F0020E0C6E09DF0EEF02F0C1
:10040C00040E0C6EE4DE0EEF02F0080E0C6EEBDE4A
:02041C001200CC
:10041E000B800BAE1BEF02F0026A0AAEFF0E026EED
:0C042E00016E006E0A360232FF0E120052
:0A043A00C582C5A201D0FDD7120053
:0E044400570E0D6E0D2EFED7000000001200A8
:10045200086A096A100E0C6E013408360936045017
:10046200085E0550D8A0053C095ED8B007D00450FC
:1004720008260550D8B0053C0926D890003601362A
:060482000C2EEAD7120067
:100488009E962EC4C9FFC7A401D0FDD79EB601D041
:10049800FDD7C5BC02D0006A03D0C584020E006E29
:0204A800120040
:1004AA000C6A0E6A0250D8A46EEF02F001C002F084
:1004BA0000C001F0006A0E860250D8A46EEF02F066
:1004CA0001C002F0016A0E960E880250D8B480EF7D
:1004DA0002F00E50035ED8A4D8A085EF02F0D8909F
:1004EA0002BE8AEF02F0003601360236032E75EF9D
:1004FA0002F085EF02F0010E0C6E76DE8DEF02F04F
:10050A00020E0C6E78DE8DEF02F0040E0C6E80DEA9
:02051A001200CD
:10051C0004012E6B2F6B2F51120802E12E518E0805
:10052C0008E379DE005201E004D004012E4B2F2B9E
:10053C00F2D70401120E2F5D02E18F0E2E5D03E344
:10054C007B0E006E05D0C580C5A001D0FDD7006A1A
:02055C0012008B
:08055E000B6A0B86FF0E120070
:1005660030C4F6FF31C4F7FF32C4F8FF0900F5CFF7
:1005760000F0005218E030C4F6FF31C4F7FF32C471
:10058600F8FF0900F5CF00F02EC4E1FF2FC4E2FF0B
:1005960000C0E6FF04012E4B2F2B010E3027000E64
:1005A60031233223DDD72EC4E1FF2FC4E2FFE66AF2
:0205B600120031
:1005B800025006180E6E086A096A0B6A035007642F
:1005C800CFEF03F006500A6E068E028E03500B6EB4
:1005D8000750036E000E0B641FEF03F00B50075E0D
:1005E800D8B4C0EF03F0070E07648EEF03F0075E80
:1005F80000C008F001C000F002C001F0026A074E16
:10060800C0EF03F0076463EF03F0075E00C008F073
:1006180001C000F0016A074EC0EF03F0076441EF24
:1006280003F0075E00C008F0006A074EC0EF03F051
:10063800076428EF03F00AC002F005C001F004C007
:1006480000F0086AE9EF04F0030E076433EF03F0E3
:10065800075E08380F0B086E074EC0EF03F0D890FE
:100668000832074EC0EF03F0D8900832074EC0EFAB
:1006780003F0D8900832C0EF03F0030E076452EF7E
:1006880003F0075E08380F0B086E0038F00B0826D9
:1006980000380F0B006E074EC0EF03F0D890003201
:1006A8000832074EC0EF03F0D89000320832074EE8
:1006B800C0EF03F0D89000320832C0EF03F0030E09
:1006C80007647AEF03F0075E08380F0B086E0038EE
:1006D800F00B082600380F0B006E0138F00B0026CF
:1006E80001380F0B016E074EC0EF03F0D8900132AE
:1006F80000320832074EC0EF03F0D89001320032C2
:100708000832074EC0EF03F0D890013200320832A9
:10071800C0EF03F0030E0764ABEF03F0075E083881
:100728000F0B086E0038F00B082600380F0B006E10
:100738000138F00B002601380F0B016E0238F00B60
:10074800012602380F0B026E074EC0EF03F0D89057
:100758000232013200320832074EC0EF03F0D8905F
:100768000232013200320832074EC0EF03F0D8904F
:100778000232013200320832096A000E0EAEB4EFBE
:1007880004F0081E001E011E021E082A0022012273
:100798000222B4EF04F00750D8A4D5EF03F0E9EF34
:1007A80004F0096A02C00AF0028E068E0750035C44
:1007B800076ED8B4A7EF04F0070E076475EF04F0CE
:1007C800075E0450096E0550046E0650056E066AF1
:1007D800074EA7EF04F0070E07644AEF04F0075E20
:1007E8000450096E0550046E056A074EA7EF04F021
:1007F800070E076428EF04F0075E0450096E046AC8
:10080800074EA7EF04F0070E07640FEF04F00AC0C5
:1008180002F0E9EF04F0030E07641AEF04F0075E34
:1008280009380F0B096E074EA7EF04F0D89009326C
:10083800074EA7EF04F0D8900932074EA7EF04F04F
:10084800D8900932A7EF04F0030E076439EF04F0DB
:10085800075E09380F0B096E0438F00B09260438B7
:100868000F0B046E074EA7EF04F0D890043209323C
:10087800074EA7EF04F0D89004320932074EA7EFCD
:1008880004F0D89004320932A7EF04F0030E07648D
:1008980061EF04F0075E09380F0B096E0438F00B9E
:1008A800092604380F0B046E0538F00B04260538AA
:1008B8000F0B056E074EA7EF04F0D89005320432EF
:1008C8000932074EA7EF04F0D890053204320932F6
:1008D800074EA7EF04F0D890053204320932A7EF8B
:1008E80004F0030E076492EF04F0075E09380F0B5B
:1008F800096E0438F00B092604380F0B046E05380E
:10090800F00B042605380F0B056E0638F00B05268C
:1009180006380F0B066E074EA7EF04F0D890063284
:10092800053204320932074EA7EF04F0D890063298
:10093800053204320932074EA7EF04F0D890063288
:10094800053204320932086A000E0EAEB4EF04F024
:10095800091E041E051E061E092A04220522062257
:100968000950082604500022055001220650022290
:100978000EBECBEF04F0D8A0DAEF04F00232013259
:1009880000320832033EDAEF04F0E4EF04F0D8B0A6
:10099800DFEF04F0000E081E001E011E021E082ACA
:1009A8000022012202220A7EDFEF04F0010E0C6E03
:1009B80041DCEBEF04F0020E0C6E3CDCEBEF04F0D4
:1009C800040E0C6E06DCEBEF04F0000E0C6E120049
:1009D8002EC402F02FC403F002C000F003C001F0DF
:1009E800024A032A00C0E9FF01C0EAFFEE5201E013
:1009F800F3D704012E51025C006E2F510358016E8B
:0A0A0800010E005E000E015A1200FC
:100A120032C400F004013207005228E02EC4E9FF7C
:100A22002FC4EAFFEE50000A0CE02EC4E9FF2FC4E7
:100A3200EAFF30C4D9FF31C4DAFFEE50DE1801E11B
:100A42000FD02EC4E9FF2FC4EAFF30C4D9FF31C44E
:100A5200DAFFDE50EE5C006E016A000E015A08D029
:100A620004012E4B2F2B304B312BD2D7006A016A57
:020A7200120070
:0E0A7400ADB202D00000FCD72EC4AEFF1200BF
:040A8200C584120015
:100A86002EC4E9FF2FC4EAFFEE500401301905E138
:100A96002EC400F02FC401F010D02EC400F02FC4D5
:100AA60001F02E4B2F2B00C0E9FF01C0EAFFEECF6D
:0C0AB60000F00052E5E1006A016A120045
:0E0AC200A8B202D00000FCD72EC4A9FF12007B
:100AD00014C4F6FF15C4F7FF16C4F8FF0900F5CFDC
:100AE00000F0005211E014C4F6FF15C4F7FF16C45D
:100AF000F8FF0900F5CF2EF4BDDF010E0401142725
:0A0B0000000E15231623E4D712009F
:100B0A000401186B050E185D0AE218511625E16EEC
:100B1A00000E1721E26E200EE66E182BF3D718513D
:100B2A001625E16E000E1721E26EE66A18071851C3
:100B3A001625196F000E17211A6F0A0E046E000E81
:100B4A00056E14C400F015C401F07EDC08C000F084
:100B5A0009C001F0300E002619C4E1FF1AC4E2FFF1
:100B6A0000C0E6FF0A0E046E000E056E14C400F003
:100B7A0015C401F069DC00C014F401C015F4000EBC
:100B8A00011802E1000E001801E102D01807CFD7C0
:020B9A00120047
:100B9C0000C008F00150006E016A026A036A0B6A19
:100BAC000C6A016A026A036A960E036E0A6A00AE48
:100BBC00E6EF05F0081E001E082AD8B4002A0A8E9B
:100BCC0000C001F008C000F0086A026A68DC12007C
:100BDC000D0E04012E6F48DF0A0E04012E6F44DF48
:020BEC001200F5
:100BEE0014C4F6FF15C4F7FF16C4F8FF0900F5CFBD
:100BFE0000F0005211E014C4F6FF15C4F7FF16C43E
:100C0E00F8FF0900F5CF2EF455DF010E040114276D
:0A0C1E00000E15231623E4D7120080
:100C280079DC9BC02EF42CDC04012E6B29DC000E31
:100C3800006E04011751005C02E11651100804E22D
:100C4800100E166F000E176F0ED01651800F2E6FF4
:100C58002E0716DC16D004011651C00F2E6F2E0772
:100C68000FDC0FD00ED0000E0401151902E1010EA1
:100C78001419EBE0000E151902E1020E1419EBE04D
:100C8800F1D71DEC02F09BC02EF444EC02F0400EAC
:100C980004012E6F44EC02F004011A6B1B6B18C49C
:100CA800E9FF19C4EAFFEE5219E018C4D9FF19C4C4
:100CB800DAFFDE50800F2E6F44EC02F00401184B6F
:100CC800192B1A4B1B2B800E006E800E1B19005C13
:100CD80002E11A51100801E201D0E1D7CEDE12007C
:100CE80019DC9BC02EF444EC02F004012E6B44EC9A
:100CF80002F0020E04012E6F44EC02F00DD0800EBB
:100D080004012E6F44EC02F015D0C00E04012E6FC2
:100D180044EC02F00FD00ED0000E0401151902E1C8
:100D2800010E1419ECE0000E151902E1020E141957
:100D3800ECE0F1D71DEC02F09BC02EF444EC02F07D
:100D4800400E04012E6F44EC02F00301276B286B60
:100D5800000E285D02E1270E275D09E2A00E0401BE
:100D68002E6F44EC02F00301274B282BF1D71DEC22
:100D780002F09BC02EF444EC02F004012E6B44EC0C
:100D880002F00DD0800E04012E6F44EC02F015D055
:100D9800C00E04012E6F44EC02F00FD00ED0000EEE
:100DA8000401151902E1010E1419ECE0000E1519E1
:0E0DB80002E1020E1419ECE0F1D75FDE12002A
:080DC600067EDCEC02F01200D5
:100DCE00000E0401151902E1000E141934E014C4CA
:100DDE00E9FF15C4EAFFEE522EE016C42EF417C436
:100DEE002FF4F3DD00C032F414C42EF415C42FF426
:100DFE0016C430F417C431F405DE000E011802E1FA
:100E0E00000E001805E114C400F015C401F015D051
:100E1E00010E040114252E6F000E15212F6F16C41E
:100E2E00E9FF17C4EAFFEECF30F426DE00C014F45B
:0C0E3E0001C015F4C5D7006A016A12005B
:100E4A000050086E0150006E016A026A036A0B6A5A
:100E5A000C6A960E036E0A6A00C001F008C000F020
:0A0E6A00086A026A55EC02F012005B
:100E7400086A096A000E07620364BFEF07F00250B4
:100E840006180A6E075003267E0ED8A050EF07F00E
:100E9400035ED8B0C4EF07F054EF07F0035ED8A0A8
:100EA400C9EF07F0028E068E02C00EF001C00BF0EF
:100EB40000C00DF000500402F4CF0CF00150050204
:100EC400F4CF00F0F3CF08F00402F3500C26F450F2
:100ED4000822000E00220D500502F3500C26F45097
:100EE4000822000E002202500402F3500826F45097
:100EF400002202500502016A000E0122F35000266E
:100F0400F45001220D500602F3500826F45000223A
:100F1400026A000E012202220B500602F350002640
:100F2400F4500122000E02220E500602F350012654
:100F3400F450022202BEA7EF07F00836003601364D
:100F440002360306D8B4C9EF07F0BAEF07F0D88029
:100F5400800E08640030000E002201220222D8A074
:100F6400BAEF07F0023201320032034AC4EF07F04D
:100F74000AAE029E000ECCEF07F0010EF9EC00F071
:100F8400CCEF07F0020EEDEC00F0CCEF07F0040E0E
:060F940000EC01F0120068
:100F9A000A6A0350D8A40A800750D8A40A820A50C1
:100FAA00D8B430EF08F0030AD8B4E9EF07F00AB072
:100FBA00E4EF07F006AE2EEF08F02CEF08F002AED1
:100FCA002CEF08F02EEF08F00250800B0A6E029EFA
:100FDA000650800B069E0A18D8B4FAEF07F00A509A
:100FEA00D8B42CEF08F02EEF08F00750035CD8B401
:100FFA0004EF08F0D8A020EF08F026EF08F006501A
:10100A00025CD8B40EEF08F0D8A020EF08F026EF63
:10101A0008F00550015CD8B418EF08F0D8A020EF0A
:10102A0008F026EF08F00450005CD8B430EF08F05E
:10103A00D8B026EF08F00A52D8B42EEF08F02CEFF9
:10104A0008F00A52D8B42CEF08F02EEF08F0D88036
:0E105A001200D8901200D880D8841200120024
:10106800C26A070EC16EC18E14C400F0003600902B
:10107800003600900050C212C28022EC02F0C282F8
:10108800C2A201D0FDD7C4CF01F0006AC35000123C
:08109800000E0112C2901200CB
:1010A0000B6A0350D8B496EF08F002500A6E028E15
:1010B0008E0E035E03AE9AEF08F0036C080E035C1D
:1010C000D8A075EF08F0036E013602C001F0026A85
:1010D000080E035CD8A075EF08F0036E0136016AB4
:1010E0000350D8A4D8907FEF08F00350D8B47FEF16
:1010F00008F0D89002320132032E79EF08F00BBCD1
:1011000001A08CEF08F0D8A08CEF08F0012AD8B429
:10111000022A02BEA9EF08F00AAEAFEF08F0021EE5
:10112000011E012AD8B4022AAFEF08F0026A016A50
:10113000AFEF08F00B800BAEB3EF08F0026A0AAE17
:10114000B3EF08F0FF0E026E016E0A360232B3EF03
:1011500008F0010E0C6E0FEC02F0B5EF08F0000E77
:101160000C6EB5EF08F0FF0E0C6E0150006E0250D1
:04117000016E1200FA
:101174000450000A12E10550000A0FE10650000A6B
:101184000CE10750000A09E1FF0E006EFF0E016E2C
:101194007F0E026EFF0E036EA8D0086A096A07501C
:1011A400D8B465EF09F00350D8B46AEF09F00250DF
:1011B40006180A6E028E068E0E6A02C008F001C07E
:1011C4000CF000C00DF004500D5E0550D8A0053C95
:1011D4000C5E0650D8A0063C085E086A0C6A0D6ACC
:1011E400D8A0FCEF08F0D890023201320032083265
:1011F400010E0E6E0750035ED8A009EF09F07E0EB3
:101204000E240326D8B06FEF09F00FEF09F07E0E1D
:101214000E240326D8A074EF09F0180E0B6E0D36B9
:101224000C3608360036013602360E360450005E9F
:101234000550D8A0053C015E0650D8A0063C025ECD
:1012440006340E120EA02AEF09F00D8035EF09F0D6
:10125400045000260550D8B0053C01260650D8B0ED
:10126400062802260D900B2E11EF09F05BEF09F012
:10127400D8900036013602360E360450005E055012
:10128400D8A0053C015E0650D8A0063C025E063498
:101294000E10010B0D26D8B00C2AD8B4082AD8A4F5
:1012A4005BEF09F008320C320D32032AD8B46FEF29
:1012B40009F00AAE089E0850026E0C50016E0D50E3
:1012C400006E77EF09F0010EAFEC02F077EF09F052
:1012D400020EF9EC00F077EF09F0040EEDEC00F0EB
:0C12E40077EF09F0080E00EC01F012009A
:1012F0000401176B14C4E9FF15C4EAFFEECF16F41E
:101300001651000A0FE016C42EF43AEC05F0040161
:10131000172B17511425E96E000E1521EA6EEECF3A
:0613200016F4EED71200E6
:10132600086A080E0C6E003408360450085ED8B001
:0E13360002D00826D89000360C2EF5D71200F3
:10134400A39A0001696B6A6B010E6A5D02E1000EEB
:10135400695D0AE2400E6925E16E010E6A21E26EC2
:10136400E66A694B6A2BF0D7636B646B696B6A6BD3
:10137400AACFD2F20201D26B2B6A2C6AA38A120082
:101384001B0E04012E6F040E2F6F18C430F419C401
:1013940031F41AC432F4B3EC02F08EEC02F09BC0C8
:1013A4002EF444EC02F004012E6B44EC02F0000E27
:1013B400006E04011751005C02E11651100804E2AA
:1013C400100E166F000E176F10D01651800F2E6F6F
:1013D4002E0744EC02F017D004011651C00F2E6FF3
:1013E4002E0744EC02F00FD00ED0000E04011519A4
:1013F40002E1010E1419E9E0000E151902E1020ED2
:101404001419EAE0F1D71DEC02F09BC02EF444EC71
:1014140002F0400E04012E6F44EC02F004012C6B28
:101424002D6B18C4F6FF19C4F7FF1AC4F8FF09009E
:10143400F5CF00F0005221E018C4F6FF19C4F7FFFD
:101444001AC4F8FF0900F5CF00F00050800F2E6F8A
:1014540044EC02F0010E04011827000E19231A238C
:101464002C4B2D2B800E006E800E2D19005C02E19A
:101474002C51100801E201D0D4D741EC05F0120040
:1014840001C404F002C405F004010551061124E06E
:10149400010E055F000E065B04C002F005C003F0F8
:1014A400044A052A03C400F004C401F0034B042BCE
:1014B40000C0E9FF01C0EAFF02C0E1FF03C0E2FF90
:1014C400EECFE6FF02C0E9FF03C0EAFFEECF00F073
:1014D400005201E101D0D8D705C400F006C401F0E0
:1014E400010E055F000E065B0050011008E004C009
:1014F400E1FF05C0E2FFE66A044A052AEDD701C40C
:0815040000F002C401F0120026
:10150C000301FF6BFCC3E9FFFDC3EAFFEECFFEF363
:10151C00FE51000A0FE0FEC32EF461EC05F003014E
:10152C00FF2BFF51FC25E96E000EFD21EA6EEECF7C
:06153C00FEF3EED71200E1
:10154200220E0C6E086A096A0A6A0B6A0C06D8B483
:101552001FD0D8900B320A320932083203320232DB
:1015620001320032D8A0F2D70C06D8B409D0045008
:1015720008260550092206500A2207500B22EAD7F4
:10158200045008260550092206500A2207500B2251
:02159200120045
:101594000B6A0A6A096A086A0E6A03340836045038
:1015A400085E0550D8A0053C095E0650D8A0063C4C
:1015B4000A5E0750D8A0073C0B5EE86AD8A0010E6B
:1015C4000E5E0336070E0C6E0334083609360A36EF
:1015D4000B360E36045003A012D0085E0550D8A076
:1015E400053C095E0650D8A0063C0A5E0750D8A008
:1015F400073C0B5EE86AD8A0010E0E5E11D00826E7
:101604000550D8B0053C09260650D8B0063C0A2639
:101614000750D8B0073C0B26E86AD8B0010E0E2656
:1016240003360C2ED1D70234083609360A360B3667
:101634000E36045003A012D0085E0550D8A0053C15
:10164400095E0650D8A0063C0A5E0750D8A0073CA5
:101654000B5EE86AD8A0010E0E5E11D00826055074
:10166400D8B0053C09260650D8B0063C0A260750D7
:10167400D8B0073C0B26E86AD8B0010E0E26023615
:10168400070E0C6E0234083609360A360B360E364F
:10169400045002A012D0085E0550D8A0053C095E93
:1016A4000650D8A0063C0A5E0750D8A0073C0B5E43
:1016B400E86AD8A0010E0E5E11D008260550D8B0F5
:1016C400053C09260650D8B0063C0A260750D8B077
:1016D400073C0B26E86AD8B0010E0E2602360C2E03
:1016E400D1D70134083609360A360B360E36045083
:1016F40002A012D0085E0550D8A0053C095E065031
:10170400D8A0063C0A5E0750D8A0073C0B5EE86AE6
:10171400D8A0010E0E5E11D008260550D8B0053CA5
:1017240009260650D8B0063C0A260750D8B0073C14
:101734000B26E86AD8B0010E0E260136070E0C6E91
:101744000134083609360A360B360E36045001A029
:1017540012D0085E0550D8A0053C095E0650D8A0FA
:10176400063C0A5E0750D8A0073C0B5EE86AD8A086
:10177400010E0E5E11D008260550D8B0053C09268E
:101784000650D8B0063C0A260750D8B0073C0B26B2
:10179400E86AD8B0010E0E2601360C2ED1D70034DB
:1017A400083609360A360B360E36045001A012D01C
:1017B400085E0550D8A0053C095E0650D8A0063C3A
:1017C4000A5E0750D8A0073C0B5EE86AD8A0010E59
:1017D4000E5E11D008260550D8B0053C09260650E7
:1017E400D8B0063C0A260750D8B0073C0B26E86A56
:1017F400D8B0010E0E260036070E0C6E00340836E3
:1018040009360A360B360E36045000A012D0085E94
:101814000550D8A0053C095E0650D8A0063C0A5ED7
:101824000750D8A0073C0B5EE86AD8A0010E0E5EF4
:1018340011D008260550D8B0053C09260650D8B06A
:10184400063C0A260750D8B0073C0B26E86AD8B0F5
:10185400010E0E2600360C2ED1D700B00ED0045047
:1018640008260550D8B0053C09260650D8B0063CD9
:0C1874000A260750D8B0073C0B261200D3
:101880000301FF6B030EFF5D0AE2FF51FD25E16ED0
:10189000000EFE21E26E200EE66EFF2BF3D7FF5105
:1018A000FD25E16E000EFE21E26EE66AFF07FF51A4
:1018B000FD250401006F000E0301FE210401016FEC
:1018C0000A0E046EFCC300F02EDD08C000F0300EDE
:1018D000002600C4E1FF01C4E2FF00C0E6FF0A0EDB
:1018E000046EFCC300F01FDD00C0FCF30050000AD2
:0C18F00001E103D00301FF07DAD712006A
:1018FC0023DDFCC314F4FDC315F4FEC316F4F7EC9E
:10190C0005F0D60E0B6E110E0C6EE40E0D6E0D2E38
:10191C00FED70C2EFCD70B2EFAD70000400E04017C
:10192C00146F010E156FDEDC0301FF5353E0090E3B
:10193C0004012E6F3AEC05F0400E0401146F010EF9
:10194C00156F410E166F000E176FE7EC06F0000EC8
:10195C00026E0150025C02E10050000803E201013A
:10196C003E4B3F2B3EC114F43FC115F425C316F476
:10197C0026C317F485EC05F0020E146F000E156FDC
:10198C00010E166F000E176F8A0E186F540E196F1A
:10199C00000E1A6FF1DC020E146F000E156F070E9D
:1019AC00166F000E176F25C318F426C319F414EC28
:1019BC0006F0C20E146F560E156F000E166F68EC03
:1019CC0005F025C314F426C315F48CDC090E2E6F18
:0A19DC003AEC05F0EEEC05F0120005
:1019E6009E96C5869EB601D0FDD7C9CF01F00301EC
:1019F600FC51000A02E1C58A01D0C59A9E96C588A7
:0C1A06009EB601D0FDD701C000F0120018
:101A1200FCC304F0FDC305F004C002F005C003F0EE
:101A2200044A052AFEC300F0FFC301F00301FE4B86
:101A3200FF2B00C0E9FF01C0EAFF02C0E1FF03C0C3
:101A4200E2FFEECFE6FF02C0E9FF03C0EAFFEE527B
:0E1A520001E0E2D7FCC300F0FDC301F012007A
:101A6000020E0401146F000E156F74EC06F0010EE7
:0E1A70000401146F000E156F74EC06F01200E6
:101A7E0004010751000806E3070E0301FC6F000E78
:101A8E00FD6F16D004010751160806E2170E03016A
:101A9E00FE6F000EFF6F08D004010751010F030106
:101AAE00FE6FFF6B000EFF23FEC3FCF3FFC3FDF3BF
:101ABE00FCC30EF4FDC30FF40401086B096B046A3A
:101ACE00056A066A076A01C400F002C401F003C485
:101ADE0002F004C403F0CDEC07F0010ED8B0000EF6
:101AEE00006E005209E005C4E1FF06C4E2FF2D0EB0
:101AFE00E66E054B062B037F01C404F002C405F00D
:101B0E0003C406F004C407F0006A016A026A036A9D
:101B1E00CDEC07F0010ED8B0000E006E005237E08B
:101B2E00000E046E000E056E000E066E7F0E076E22
:101B3E0001C400F002C401F003C402F004C403F0B7
:101B4E00CDEC07F0010ED8B0000E006E00521FE073
:101B5E0001C400F002C401F003C402F004C403F097
:101B6E00000E046E000E056E200E066E820E076EBF
:101B7E003AEC07F000C001F401C002F402C003F415
:101B8E0003C004F4010E085F000E095BC9D7000EF6
:101B9E00046E000E056E200E066E820E076E01C4D8
:101BAE0000F002C401F003C402F004C403F0CDEC53
:101BBE0007F0000ED8B0010E006E00521EE0000EAF
:101BCE00046E000E056E200E066E820E076E01C4A8
:101BDE0000F002C401F003C402F004C403F0BAEC36
:101BEE0008F000C001F401C002F402C003F403C007
:101BFE0004F40401084B092BCAD708510E270951CA
:101C0E000F23010E0A6F000E0B6F000E106F000EE9
:101C1E00116F000E126F7F0E136F800E0B19006E78
:101C2E00800E0F19005C02E10E510A5D1EE2000EDD
:101C3E00046E000E056E200E066E820E076E10C428
:101C4E0000F011C401F012C402F013C403F0BAEC98
:101C5E0008F000C010F401C011F402C012F403C069
:101C6E0013F404010A4B0B2BD8D7000E046E000E92
:101C7E00056E000E066E800E076E10C400F011C4C5
:101C8E0001F012C402F013C403F0BAEC08F001C460
:101C9E0004F002C405F003C406F004C407F0DCEC43
:101CAE0002F000C001F401C002F402C003F403C04C
:101CBE0004F4000E046E000E056E200E066E820EEB
:101CCE00076ECDEC07F0000ED8B0010E006E00527C
:101CDE000BE0000E0401016F000E026F000E036F89
:101CEE007F0E046F084B092B0401800E0919006E3C
:101CFE00800E005C02E1000E085D38E205C4E1FFD3
:101D0E0006C4E2FF300EE66E054B062B05C4E1FF5E
:101D1E0006C4E2FF2E0EE66E054B062B800E0F1943
:101D2E00006E800E005C02E1000E0E5D04E20E51AC
:101D3E00085F0F51095BFF0E0A6FFF0E0B6F800ECF
:101D4E000919006E800E0B19005C02E10A51085D44
:101D5E000DE205C4E1FF06C4E2FF300EE66E054B50
:101D6E00062B010E0A5F000E0B5BE9D70A6B0B6B9D
:101D7E00800E0B19006E800E0F19005C02E10E51E1
:101D8E000A5D63E201C400F002C401F003C402F074
:101D9E0004C403F050EC08F000C00CF401C00DF4C4
:101DAE00300E002605C4E1FF06C4E2FF00C0E6FFC8
:101DBE00054B062B0B51091902E108510A1908E1CE
:101DCE0005C4E1FF06C4E2FF2E0EE66E054B062BA0
:101DDE000CC400F00DC401F0CEEC05F000C010F400
:101DEE0001C011F402C012F403C013F400C004F0D9
:101DFE0001C005F002C006F003C007F001C400F0F8
:101E0E0002C401F003C402F004C403F0E3EC06F0D4
:101E1E0000C001F401C002F402C003F403C004F4D4
:101E2E00000E046E000E056E200E066E820E076EFC
:101E3E003AEC07F000C001F401C002F402C003F452
:101E4E0003C004F40A4B0B2B93D705C4E1FF06C461
:061E5E00E2FFE66A12003B
:101E6400FCC304F0FDC305F004C0E9FF05C0EAFFAC
:101E7400EE5203E0044A052AF7D704C002F005C075
:101E840003F0044A052AFEC300F0FFC301F0030176
:101E9400FE4BFF2B00C0E9FF01C0EAFF02C0E1FFD7
:101EA40003C0E2FFEECFE6FF02C0E9FF03C0EAFF92
:101EB400EE5201E0E2D7FCC300F0FDC301F01200D2
:101EC400800E0301FD6FFE6BFF6B300E0401006F8B
:101ED400300E016F300E026F300E036F300E046F40
:101EE400300E056F300E066F300E076F086B800ED4
:101EF4000301FF19006E800E005C02E1080EFE5D16
:101F040013E2FD51FC15016E0150000808E2000EB9
:101F1400FE25E16E040EFF21E26E310EE66EFD3306
:101F2400FD9FFE4BFF2BE3D70401086B000E006EF0
:061F3400040E016E120014
:101F3A00020E0401146F34EC08F0060E005C056E04
:101F4A00000E0158066E05C088F206C089F2070E17
:101F5A0002018615036E87C204F0000E041603C040
:101F6A0000F004C001F0003600900136760E00241D
:101F7A00E16E020E0120E26E05C0E6FF06C0E6FF32
:101F8A00864B872B01013C6B3D6B0301276B286B4A
:101F9A00000E285D02E1080E275D16E227C300F055
:101FAA0028C301F0003600900136760E0024D96E5F
:101FBA00020E0120DA6EDE5001013C27DE503D237D
:101FCA000301274B282BE4D73CC100F03DC101F0A7
:101FDA0025EC07F0000E046E000E056E250E066E47
:0A1FEA007A0E076E3AEC07F01200C1
:101FF4008EEC02F09BC02EF444EC02F004012E6B34
:1020040044EC02F0800E006E800E04010419005CA2
:1020140002E10351100804E2100E036F000E046F76
:1020240010D00351800F2E6F2E0744EC02F017D00E
:1020340004010351C00F2E6F2E0744EC02F00FD0A1
:102044000ED0000E0401021902E1010E0119E9E0AB
:10205400000E021902E1020E0119EAE0F1D71DECAB
:1020640002F09BC02EF444EC02F0400E04012E6FEB
:1020740044EC02F005C42EF444EC02F041EC05F00B
:02208400120048
:10208600440E0401146F550E156F000E166F68ECA2
:1020960005F0BEC3FCF3D50E0301FD6F020EFE6F05
:1020A60040EC0CF0D50E0401146F020E156F78EC9F
:1020B60009F08EEC02F0BEC32EF444EC02F00050A0
:1020C600000A0CE09E0E0401146F550E156F000EEB
:1020D600166F68EC05F00301BF6B0CD0310E0401DE
:1020E600146F560E156F000E166F68EC05F0010E94
:1020F6000301BF6F41EC05F0EEEC05F0BFC300F045
:022106001200C5
:10210800949894968B988B9694889486C79EC79C2F
:06211800380EC66E120035
:10211E00FF0E03011B6FFF0E1C6FFF0E1D6FFF0ED8
:0E212E001E6FC26A070EC16EC18EC280120003
:10213C00FF0E986EEF0E926EBF0E946EC088F90E65
:10214C00C16EFF0EC26EC09893809384928095945A
:10215C00988693869596F19E9A8A92988988958E00
:0E216C00998695989698959C8C988D9812005F
:10217A000900F5CFE6FF0006FBE10106F9E11200CE
:10218A000301C46BC56B000EC55D02E10A0EC45D96
:10219A000BE2C451C225E16EC551C321E26E200E85
:1021AA00E66EC44BC52BEFD7C451C225E16EC551AB
:1021BA00C321E26EE66A010EC45F000EC55BC4511C
:1021CA00C225C66FC551C321C76F0A0E046E000E21
:1021DA00056E066E076EBEC300F0BFC301F0C0C332
:1021EA0002F0C1C303F0CAEC0AF008C000F009C04B
:1021FA0001F00AC002F00BC003F0300E0026C6C37D
:10220A00E1FFC7C3E2FF00C0E6FF0A0E046E000E3C
:10221A00056E066E076EBEC300F0BFC301F0C0C3F1
:10222A0002F0C1C303F0CAEC0AF000C0BEF301C059
:10223A00BFF302C0C0F303C0C1F3000E046E03185B
:10224A0008E10450021805E10450011802E10050A7
:10225A00000A01E105D0010EC45F000EC55BAFD7CD
:02226A00120060
:10226C00C20E0301156F0A0E166F2E0E176F040E99
:10227C00186FFF0EBA6FFF0EBB6F000EBC6F000E17
:10228C00BD6FFF0EB06FFF0EB16F000EB26F000E80
:10229C00B36FFF0EAC6FFF0EAD6F000EAE6F000E86
:1022AC00AF6FA88A900E9C6E98849892A4AA03D0C3
:0822BC00AACF00F0FBD71200CD
:1022C400740E0301156F0A0E166F2E0E176F040E8F
:1022D400186FFF0EBA6FFF0EBB6F000EBC6F000EBF
:1022E400BD6FFF0EB06FFF0EB16F000EB26F000E28
:1022F400B36FFF0EAC6FFF0EAD6F000EAE6F000E2E
:10230400AF6FAD8A900EAC6E948E949C9EAA03D04F
:08231400AFCF00F0FBD712006F
:10231C00010E0401146F000E156F74EC06F02A0EFA
:10232C000301256F030E266F25C32EF426C32FF44D
:10233C00BB0E0401306F560E316F000E326FB3ECD2
:10234C0002F01FC301F420C302F421C303F422C31F
:10235C0004F4D50E0401056F020E066F020E076F12
:10236C003FEC0DF025C3FCF326C3FDF3D50E0301A2
:10237C00FE6F020EFF6F70DD25C32EF426C32FF403
:10238C00ECEC04F000C027F301C028F372C2FCF39C
:10239C00D50E0301FD6F020EFE6F40EC0CF025C351
:1023AC00FCF326C3FDF3D50E0301FE6F020EFF6F87
:1023BC0053DD100E2525E16E000E2621E26EE66A35
:1023CC00010E0401146F000E156F010E166F000E36
:1023DC00176F25C318F426C319F414EC06F0D50EA8
:1023EC002E6F020E2F6F790E306F540E316F000E60
:1023FC00326FB3EC02F0000E80B0010E0201D86F08
:10240C00300ED827000E030129B5010E0201DE6F34
:10241C00300EDE27000E030129BB010E0201E36F13
:10242C00300EE327E56B020E0401146F000E156FDE
:10243C0074EC06F0020E0401146F000E156F010E01
:10244C00166F000E176FD50E186F020E196F14EC65
:04245C0006F0120074
:10246000D596D584D582D580D59AD59C480ED76E81
:10247000E50ED66EF2940301B86BB96BAA6BAB6B29
:08248000F184F28AD58E1200EE
:102488008EEC02F0400E04012E6F44EC02F0120EA6
:1024980004012E6F44EC02F0BEC32EF444EC02F0AB
:0624A80041EC05F01200FA
:1024AE00670E0401146F510E156F000E166F68EC57
:1024BE0005F0BEC314F4BFC315F478EC09F0EEECCE
:1024CE0005F0A2EC09F02A0E0401146F520E156FDE
:1024DE00000E166F68EC05F0010E0401146F000E6D
:1024EE00156F010E166F000E176FBD0E186F540E7E
:1024FE00196F000E1A6FC2EC09F00F0E006E000E6F
:10250E00016E026E036E74C204F075C205F0000E09
:10251E00020175BFFF0E066E076EA1EC0AF0A70E44
:10252E0000240401146F4E0E0120156F000E0220C0
:10253E00166F68EC05F0EEEC05F0420E04012E6FFE
:10254E00020E2F6F6A0E306F560E316F000E326F05
:10255E00B3EC02F04A0E04012E6F020E2F6F0F0E17
:10256E00006E000E016E026E036E74C204F075C230
:10257E0005F0000E020175BFFF0E066E076EA1EC90
:10258E000AF0A70E00240401306F4E0E0120316FA9
:10259E00000E0220326FB3EC02F0020E0401146F33
:1025AE00000E156F74EC06F0020E0401146F000E8F
:1025BE00156F010E166F000E176F0F0E006E000EC8
:1025CE00016E026E036E74C204F075C205F0000E49
:1025DE00020175BFFF0E066E076EA1EC0AF0A70E84
:1025EE0000240401186F4E0E0120196F000E0220F8
:1025FE001A6FC2EC09F0420E0301FC6F020EFD6F62
:10260E0086EC0AF00D0E04012E6F61EC05F0A2ECC3
:10261E0009F0B70E0B6EA10E0C6EC30E0D6E0D2EC5
:10262E00FED70C2EFCD70B2EFAD700000000400E62
:10263E000401146F010E156F78EC09F03E0E0101C6
:10264E00406FA2EC09F0A30E0401146F510E156F2A
:10265E00000E166F68EC05F025C3FCF326C3FDF3E0
:10266E0086EC0AF00D0E04012E6F61EC05F00A0ED9
:10267E0004012E6F61EC05F01A0E04012E6F61EC51
:10268E0005F0A2EC09F0020E0A6E120E0B6EF20E9F
:10269E000C6E240E0D6E0D2EFED70C2EFCD70B2EAF
:1026AE00FAD70A2EF8D70000400E0401146F010E5F
:1026BE00156F78EC09F0400E146F010E156F310E88
:1026CE00166F000E176FE7EC06F000C040F201C067
:1026DE0041F2000E026E0150025C02E10050000851
:1026EE000AE2440E0401146F520E156F000E166F9F
:1026FE0068EC05F064D0400E0401146F010E156FE6
:10270E00370E166F000E176FE7EC06F000C040F2A2
:10271E0001C041F2000E026E0150025C02E1005057
:10272E0000084DE2540E0401146F550E156F000E85
:10273E00166F68EC05F0400E0401146F010E156F54
:10274E003A0E166F000E176FE7EC06F000C040F25F
:10275E0001C041F225C301F426C302F400C003F404
:10276E0001C004F40A0E0401056F000E066F42EC60
:10277E000AF025C314F426C315F478EC09F0EEEC38
:10278E0005F01A0E02014025E16E000E4121E26EA7
:10279E00E66A020E0401146F000E156F74EC06F05B
:1027AE00020E0401146F000E156F010E166F000E4F
:1027BE00176F25C318F426C319F414EC06F0EEECCB
:0827CE0005F0A2EC09F0120075
:1027D6002A0E0301256F030E266FBEC3E1FFBFC39A
:1027E600E2FFE66AC06BBEC32EF4BFC32FF4D00E61
:1027F6000401306F520E316F000E326FB3EC02F0EF
:10280600BEC32EF4BFC32FF4ECEC04F000C09CF062
:1028160001C09DF0030129A99FD0C06BC00E040121
:102826002E6F030E2F6FD30E306F550E316F000EC5
:10283600326FB3EC02F01AC3FCF362EC0FF000C087
:10284600FEF301C0FFF3C40E0301FC6F030EFD6F20
:1028560009EC0DF0C00E04012E6F030E2F6FECEC89
:1028660004F000C09CF001C09DF0C00E0024E16E93
:10287600030E0120E26E0D0EE66E00019C4B9D2BB1
:10288600C00E9C25E16E030E9D21E26E0A0EE66ED9
:102896009C4B9D2BC00E9C25E16E030E9D21E26E86
:1028A600E66ABEC3FCF3BFC3FDF3C00E0301FE6FB1
:1028B600030EFF6F32EC0FF0C06BC00E04012E6FDB
:1028C600030E2F6FB90E306F550E316F000E326F3B
:1028D600B3EC02F019C3FCF362EC0FF000C0FEF398
:1028E60001C0FFF3C40E0301FC6F030EFD6F09EC7C
:1028F6000DF0C00E04012E6F030E2F6FECEC04F0EA
:1029060000C09CF001C09DF0C00E0024E16E030ED5
:102916000120E26E0D0EE66E00019C4B9D2BC00E53
:102926009C25E16E030E9D21E26E0A0EE66E9C4B1F
:102936009D2BC00E9C25E16E030E9D21E26EE66A7C
:10294600BEC3FCF3BFC3FDF3C00E0301FE6F030E4F
:10295600FF6F32EC0FF00ED0C06BC00E04012E6F6D
:10296600030E2F6F010E306F540E316F000E326F53
:10297600B3EC02F00301C06BC00E04012E6F030E10
:102986002F6F840E306F560E316F000E326FB3EC20
:1029960002F0C00E04012E6F030E2F6FECEC04F054
:1029A60000C09CF001C09DF0C00E0024E16E030E35
:1029B6000120E26E006A83BE002A300E002600C0A7
:1029C600E6FF00019C4B9D2BC00E9C25E16E030E7D
:1029D6009D21E26E0D0EE66E9C4B9D2BC00E9C2536
:1029E600E16E030E9D21E26E0A0EE66E9C4B9D2B58
:1029F600C00E9C25E16E030E9D21E26EE66ABEC303
:102A0600FCF3BFC3FDF3C00E0301FE6F030EFF6FA1
:102A160032EC0FF0C06BC00E04012E6F030E2F6F49
:102A26007C0E306F560E316F000E326FB3EC02F033
:102A3600C00E04012E6F030E2F6FECEC04F000C0E5
:102A46009CF001C09DF0C00E0024E16E030E012033
:102A5600E26E006A87B6002A300E002600C0E6FF46
:102A660000019C4B9D2BC00E9C25E16E030E9D2103
:102A7600E26E0D0EE66E9C4B9D2BC00E9C25E16E04
:102A8600030E9D21E26E0A0EE66E9C4B9D2BC00E38
:102A96009C25E16E030E9D21E26EE66ABEC3FCF341
:102AA600BFC3FDF3C00E0301FE6F030EFF6F32ECD2
:102AB6000FF0C06BC00E04012E6F030E2F6F8C0E2D
:102AC600306F560E316F000E326FB3EC02F0C00E4F
:102AD60004012E6F030E2F6FECEC04F000C09CF087
:102AE60001C09DF0C00E0024E16E030E0120E26ECF
:102AF600006A83B8002A300E002600C0E6FF0001F7
:102B06009C4B9D2BC00E9C25E16E030E9D21E26E13
:102B16000D0EE66E9C4B9D2BC00E9C25E16E030EA2
:102B26009D21E26E0A0EE66E9C4B9D2BC00E9C25E7
:102B3600E16E030E9D21E26EE66ABEC3FCF3BFC3DF
:102B4600FDF3C00E0301FE6F030EFF6F32EC0FF0B4
:102B5600C06BC00E04012E6F030E2F6FA40E306FD4
:102B6600560E316F000E326FB3EC02F0C00E040148
:102B76002E6F030E2F6FECEC04F000C09CF001C02A
:102B86009DF0C00E0024E16E030E0120E26E006A85
:102B960084B8002A300E002600C0E6FF00019C4BD8
:102BA6009D2BC00E9C25E16E030E9D21E26E0D0E3F
:102BB600E66E9C4B9D2BC00E9C25E16E030E9D215F
:102BC600E26E0A0EE66E9C4B9D2BC00E9C25E16EB6
:102BD600030E9D21E26EE66ABEC3FCF3BFC3FDF39E
:102BE600C00E0301FE6F030EFF6F32EC0FF0C06BD9
:102BF600010E0401146F34EC08F000C023F301C089
:102C060024F30150020802E1005058080EE2C00EFB
:102C160004012E6F030E2F6F680E306F540E316F46
:102C2600000E326FB3EC02F00DD0C00E04012E6F11
:102C3600030E2F6FF30E306F560E316F000E326F8C
:102C4600B3EC02F0C00E04012E6F030E2F6FECECF6
:102C560004F000C09CF001C09DF023C314F424C30B
:102C660015F4C00E0024166F030E0120176F85ECB5
:102C760005F0C00E2E6F030E2F6FECEC04F000C0B3
:102C86009CF001C09DF0C00E0024E16E030E0120F1
:102C9600E26E0D0EE66E00019C4B9D2BC00E9C2530
:102CA600E16E030E9D21E26E0A0EE66E9C4B9D2B95
:102CB600C00E9C25E16E030E9D21E26EE66ABEC340
:102CC600FCF3BFC3FDF3C00E0301FE6F030EFF6FDF
:102CD60032EC0FF0C06B9DEC0FF000C01FF301C08B
:102CE60020F302C021F303C022F3C00E04012E6FAD
:102CF600030E2F6F940E306F560E316F000E326F2B
:102D0600B3EC02F0C00E04012E6F030E2F6FECEC35
:102D160004F000C09CF001C09DF01FC301F420C365
:102D260002F421C303F422C304F4C00E0024056F89
:102D3600030E0120066F020E076F3FEC0DF0C00E6A
:102D46002E6F030E2F6FECEC04F000C09CF001C058
:102D56009DF0C00E0024E16E030E0120E26EB00E5F
:102D6600E66E00019C4B9D2BC00E9C25E16E030E6A
:102D76009D21E26E430EE66E9C4B9D2BC00E9C255C
:102D8600E16E030E9D21E26EE66ABEC3FCF3BFC38D
:102D9600FDF3C00E0301FE6F030EFF6F32EC0FF062
:102DA600C06BC00E04012E6F030E2F6F270E306FFF
:102DB600560E316F000E326FB3EC02F0BEC3FCF359
:102DC600BFC3FDF3C00E0301FE6F030EFF6F32ECAF
:102DD6000FF0C06BBEC32EF4BFC32FF4ECEC04F0AF
:0A2DE60000C09CF001C09DF0120037
:102DF0009D9A00019C6B9D6B000E9D5D02E1800E13
:102E00009C5D0AE2BC0E9C25E16E000E9D21E26EE7
:102E1000E66A9C4B9D2BF0D79C6B9D6B186A196AD8
:0E2E2000AFCF1AF01A6A2D6A2E6A9D8A120030
:102E2E008EEC02F09BC02EF444EC02F0400E040136
:102E3E002E6F44EC02F00A0E04012E6F44EC02F0E9
:102E4E0004012E6B44EC02F041EC05F08EEC02F026
:102E5E00400E04012E6F44EC02F004012E6B44EC84
:102E6E0002F004012E6B44EC02F0FF0E04012E6FF3
:102E7E0044EC02F004012E6B44EC02F0FF0E040150
:102E8E002E6F44EC02F041EC05F08EEC02F0400E99
:102E9E0004012E6F44EC02F00D0E04012E6F44EC73
:102EAE0002F0FF0E04012E6F44EC02F041EC05F02F
:022EBE00120000
:102EC0000301C06BC16B1F0E0B6E710E0C6E1E0EDC
:102ED0000D6E0D2EFED70C2EFCD70B2EFAD7000050
:102EE0008EEC02F09BC02EF444EC02F000C0BEF366
:102EF000000E0301BF6F000EBF1902E1000EBE19E4
:102F000005E0C0C300F0C1C301F0E6D0C04BC12B47
:102F10000D0E0B6E2D0E0C6ED70E0D6E0D2EFED7F8
:102F20000C2EFCD70B2EFAD70000000004012E6BEC
:102F300044EC02F000C0BEF3000E0301BF6F800E30
:102F4000006E800EBF19005C02E1BE51000805E270
:102F5000C0C300F0C1C301F0BFD0C04BC12B240ED1
:102F600004012E6F44EC02F00C0E04012E6F44ECB1
:102F700002F0060E04012E6F44EC02F0250E04014F
:102F80002E6F44EC02F0060E04012E6F44EC02F0AA
:102F9000110E04012E6F44EC02F0420E04012E6F5C
:102FA00044EC02F0960E04012E6F44EC02F0240E65
:102FB00004012E6F44EC02F000C0BEF3000E0301CA
:102FC000BF6F800E006E800EBF19005C02E1BE5123
:102FD000000805E2C0C300F0C1C301F07DD0C04BC2
:102FE000C12B0C0E04012E6F44EC02F000C0BEF3A6
:102FF000000E0301BF6F800E006E800EBF19005CD3
:1030000002E1BE51000805E2C0C300F0C1C301F0F7
:1030100063D0C04BC12B060E04012E6F44EC02F0AE
:1030200000C0BEF3000E0301BF6F800E006E800E65
:10303000BF19005C02E1BE51000805E2C0C300F008
:10304000C1C301F049D0C04BC12B020E04012E6F49
:1030500044EC02F000C0BEF3000E0301BF6F800E0F
:10306000006E800EBF19005C02E1BE51000805E24F
:10307000C0C300F0C1C301F02FD0C04BC12B010E63
:1030800004012E6F44EC02F000C0BEF3000E0301F9
:10309000BF6F800E006E800EBF19005C02E1BE5152
:1030A000000805E2C0C300F0C1C301F015D0070E4F
:1030B0000B6E170E0C6E6A0E0D6E0D2EFED70C2EBB
:1030C000FCD70B2EFAD7000041EC05F0C04BC12B0A
:0A30D000C0C300F0C1C301F01200FC
:1030DA000301BE6BBF6B2F6A306A530E0401146F73
:1030EA00530E156F000E166F68EC05F0A2EC09F08E
:1030FA00100E0401146F570E156F000E166FF7ECC1
:10310A0005F03D0E0B6EE10E0C6E3F0E0D6E0D2E90
:10311A00FED70C2EFCD70B2EFAD700000000000EAB
:10312A002C1802E1010E2B1833E1400E0401146F32
:10313A00010E156F280E166F000E176FE7EC06F0DA
:10314A00000E026E0150025C02E10050000820E20B
:10315A00150E0301BE6F000EBF6F010E2F6E000E1B
:10316A00306E400E0401146F010E156F78EC09F0F1
:10317A00020E146F000E156F010E166F000E176FF8
:10318A00AC0E186F540E196F000E1A6FC2EC09F0CC
:10319A001F0E0B6E710E0C6E1E0E0D6E0D2EFED7CF
:1031AA000C2EFCD70B2EFAD700000301BE4BBF2B07
:1031BA00800EBF19006E800E005C02E1140EBE5D27
:1031CA0007E2000E301802E1000E2F1801E18ED737
:0231DA001200E1
:1031DC008EEC02F0400E04012E6F44EC02F04F0E08
:1031EC000D6E0D2EFED700000000130E04012E6F85
:1031FC0044EC02F041EC05F08EEC02F0410E0401BF
:10320C002E6F44EC02F00301FC6BF3EC0CF000C0ED
:0C321C00BEF341EC05F0BEC300F0120050
:10322800010E0401146F000E156F010E166F000ECB
:10323800176FDF0E186F540E196F000E1A6FC2EC5D
:1032480009F08D8801013E6B3F6B03012987480E09
:103258000401146F510E156F000E166F68EC05F01F
:10326800820E0301FC6F550EFD6F000EFE6F000EFF
:1032780029B7010EFF6F7EEC0CF0190E0401146FD4
:103288004E0E156F000E166F68EC05F0450E030123
:10329800FC6F560EFD6F000EFE6F000E29B7010E73
:1032A800FF6F7EEC0CF0500E0401146F4F0E156F7B
:1032B800000E166F68EC05F03B0E0301FC6F560E0E
:1032C800FD6F000EFE6F000E29B7010EFF6F7EEC3A
:1032D8000CF0290E0401146F4F0E156F000E166FB7
:1032E80068EC05F0040E0301FC6F560EFD6F000E2E
:1032F800FE6F000E29B7010EFF6F7EEC0CF07C0EFE
:103308000401146F4D0E156F000E166F68EC05F072
:10331800120E0301FC6F530EFD6F000EFE6F000EC0
:1033280029B7010EFF6F7EEC0CF05C0E0B6E510E90
:103338000C6E600E0D6E0D2EFED70C2EFCD70B2ECC
:10334800FAD70000DD0E0401146F530E156F000E3E
:10335800166F68EC05F030EC0DF0010E0401146FE7
:10336800000E156F010E166F000E176FCE0E186F38
:10337800540E196F000E1A6FC2EC09F03EC114F416
:103388003FC115F425C316F426C317F485EC05F0E0
:1033980025C314F426C315F478EC09F0020E146F53
:1033A800000E156F74EC06F0B40E0401146F560E7F
:1033B800156F000E166F68EC05F0020E0401146F0D
:1033C800000E156F010E166F000E176F9B0E186F0B
:1033D800540E196F000E1A6FC2EC09F0020E016F3D
:1033E800000E026F030E036F000E046F300E010112
:1033F8003E250401056FFAEC0FF03EC100F03FC115
:0434080001F01200BD
:10340C008AEC2BF09EEC10F08D882A0E0301256FB0
:10341C00030E266F2A6B0201D56B0101406B030171
:10342C00236B246B0201CE6BCF6BD06BD16B010184
:10343C003E6B3F6B030129872995299B298F299D79
:10344C008C9C0201746B756B8D988C88800ECA6F86
:10345C00BB0ECB6F000ECC6FCD6F800E0301BE6F19
:10346C00BB0EBF6F000EC06F000EC16F25C3C2F341
:10347C0026C3C3F3C5EC10F07E86020E7F6E700E71
:10348C00B06EAD8462EC11F00C0E04012E6F3AECB0
:10349C0005F01F0E0B6E710E0C6E1E0E0D6E0D2EAA
:1034AC00FED70C2EFCD70B2EFAD70000EEEC05F055
:1034BC008C987C86020E7D6E700EAB6EA88436ECFA
:1034CC0011F03F0E0401146F4D0E156F000E166FA8
:1034DC0068EC05F0550E0401146F4C0E156F000EC0
:1034EC00166F68EC05F0B60E0401146F4C0E156FD8
:1034FC00000E166F68EC05F0FF0E0401146F4E0EF3
:10350C00156F000E166F68EC05F0580E0401146F61
:10351C00560E156F000E166F68EC05F025C314F4EB
:10352C0026C315F478EC09F0EEEC05F0230E04013B
:10353C002E6F3AEC05F0EEEC05F0020E0A6E310E31
:10354C000B6E620E0C6E450E0D6E0D2EFED70C2EF4
:10355C00FCD70B2EFAD70A2EF8D7240E04012E6FA7
:10356C003AEC05F0EEEC05F08FEC10F0C60E040111
:10357C00146F550E156F000E166F68EC05F07C0E6F
:10358C000401146F530E156F000E166F68EC05F0E6
:10359C00780EC86E84EC10F0070E0B6E170E0C6EC6
:1035AC006A0E0D6E0D2EFED70C2EFCD70B2EFAD7F5
:1035BC0000009D0E0401146F4F0E156F000E166F58
:1035CC0068EC05F0010E0401146F34EC08F000C037
:1035DC0023F301C024F300C014F401C015F425C377
:1035EC0016F426C317F485EC05F025C314F426C392
:1035FC0015F478EC09F0090E2E6F3AEC05F0010188
:10360C003C6B3D6B020E0401146F34EC08F000C0EF
:10361C0088F201C089F200C014F401C015F425C36E
:10362C0016F426C317F485EC05F025C314F426C351
:10363C0015F478EC09F0EEEC05F00301276B286B20
:10364C00000E285D02E1080E275D14E227C300F08E
:10365C0028C301F0003600900136760E0024E16E8E
:10366C00020E0120E26E88C2E6FF89C2E6FF274BFC
:10367C00282BE6D70201866B876B000E0401146FB2
:10368C004D0E156F000E166F68EC05F0740E0001F0
:10369C009B6F100E0401146F520E156F000E166FF7
:1036AC0068EC05F09BC0BEF343EC10F00201C86B54
:1036BC00C96B00DC00C0C8F201C0C9F2070E0B6E6A
:1036CC00170E0C6E6A0E0D6E0D2EFED70C2EFCD73F
:1036DC000B2EFAD7000030EC0DF0A40E0401146F81
:1036EC00530E156F000E166F68EC05F0C8C214F47B
:1036FC00C9C215F425C316F426C317F485EC05F0DE
:10370C00750E146F520E156F000E166F68EC05F0E7
:10371C0025C314F426C315F478EC09F0EEEC05F08F
:10372C00010E0401146F000E156F74EC06F0010EFF
:10373C000401146F000E156F010E166F000E176F3B
:10374C00010E186F550E196F000E1A6FC2EC09F0AE
:10375C00290E146F510E156F000E166F68EC05F0E4
:10376C00400E0301BE6F43EC10F000C01AF017ECD2
:10377C0017F00301196B1A50010A14E1020E04012F
:10378C00146F000E156F010E166F000E176FF00EF2
:10379C00186F540E196F000E1A6FC2EC09F003016A
:1037AC00298912D02999020E0401146F000E156F8D
:1037BC00010E166F000E176F120E186F550E196F43
:1037CC00000E1A6FC2EC09F01A6A3D0E0B6EE10E78
:1037DC000C6E3F0E0D6E04010D2EFDD70C2EFBD77B
:1037EC000B2EF9D7000000006C0E146F500E156FE5
:1037FC00000E166F68EC05F03D0E0B6EE10E0C6EB4
:10380C003F0E0D6E0D2EFED70C2EFCD70B2EFAD7BD
:10381C00000000008C84020E0A6E310E0B6E620EDC
:10382C000C6E450E0D6E0D2EFED70C2EFCD70B2EEE
:10383C00FAD70A2EF8D78C943D0E0B6EE10E0C6E57
:10384C003F0E0D6E0D2EFED70C2EFCD70B2EFAD77D
:10385C00000000008C96A30E0401146F520E156F1D
:10386C00000E166F68EC05F0A2EC09F0AC8EAC867D
:10387C00AC969C96D08EA38AF28CF28E28DC000E2D
:10388C00301802E1010E2F180AE1CB0E0401146F5F
:10389C00530E156F000E166F68EC05F019D00A0E5A
:1038AC000401146F510E156F000E166F68EC05F0C5
:1038BC008C783D0E0B6EE10E0C6E3F0E0D6E0D2EC8
:1038CC00FED70C2EFCD70B2EFAD700000000F0D739
:1038DC002A0E0301256F030E266FA0DC00C03EF1FB
:1038EC0001C03FF1000E011802E1050E00180CE1B9
:1038FC00050E0401146F570E156F000E166F68EC51
:10390C0005F00301298558D0C90E0401146F560E19
:10391C00156F000E166F68EC05F003012995D40E97
:10392C000401146F4E0E156F000E166F68EC05F047
:10393C0030EC0DF0010E0401146F000E156F010E2A
:10394C00166F000E176F230E186F550E196F000EA1
:10395C001A6FC2EC09F0010E016F000E026F0F0E10
:10396C00036F000E046F300E01013E250401056F3C
:10397C00FAEC0FF0020E0401146F000E156F010E1D
:10398C00166F000E176F570E186F540E196F000E2E
:10399C001A6FC2EC09F0020E0A6E310E0B6E620E3B
:1039AC000C6E450E0D6E0D2EFED70C2EFCD70B2E6D
:1039BC00FAD70A2EF8D7B3D7EEEC05F07A0E0B6EC9
:1039CC00C10E0C6E810E0D6E0D2EFED70C2EFCD77B
:1039DC000B2EFAD7000000008FEC10F08C98E50E3F
:1039EC000401146F4F0E156F000E166F68EC05F086
:1039FC00010E0401146F34EC08F000C023F301C075
:103A0C0024F300C014F401C015F425C316F426C326
:103A1C0017F485EC05F025C314F426C315F478ECE3
:103A2C0009F0090E2E6F3AEC05F0020E0401146F2A
:103A3C0034EC08F000C088F201C089F200C014F424
:103A4C0001C015F425C316F426C317F485EC05F054
:103A5C0025C314F426C315F478EC09F0EEEC05F04C
:103A6C002A0E0301256F030E266F090E0401146F35
:103A7C00500E156F000E166F68EC05F025C3BEF3E3
:103A8C0026C3BFF3EBEC13F000C0C6F201C0C7F2C3
:103A9C00EEEC05F0070E0B6E170E0C6E6A0E0D6E2B
:103AAC000D2EFED70C2EFCD70B2EFAD700008D98BE
:103ABC0001013E6B3F6B03012997299B8C9C8C0E5B
:103ACC000401146F520E156F000E166F68EC05F0A2
:103ADC00F8EC16F00201726B736B2A0E0301256F62
:103AEC00030E266F81B413D025C32EF426C32FF4F6
:103AFC00CC0E0401306F500E316F000E326FB3ECF0
:103B0C0002F025C3BEF326C3BFF357EC12F003013A
:103B1C00299F2A0E256F030E266FF8EC16F030EC59
:103B2C0012F029A908D019C3BEF344EC12F0EEEC44
:103B3C0018F000C01AF3000E0201D11902E1000EB8
:103B4C00D019D8A476D172C214F473C215F4D50E60
:103B5C000401166F020E176F85EC05F0D50E146F6D
:103B6C00020E156F78EC09F0010E146F34EC08F0AE
:103B7C0000C023F301C024F300C014F401C015F4F9
:103B8C00D50E0401166F020E176F85EC05F0FF0EB3
:103B9C00146F560E156F000E166F68EC05F0D50EEF
:103BAC000401146F020E156F78EC09F01C0E146FE3
:103BBC00560E156F000E166F68EC05F0020E040120
:103BCC00146F34EC08F0060E005E000E015A00C0B3
:103BDC0088F201C089F200C014F401C015F4D50EAE
:103BEC000401166F020E176F85EC05F0D50E146FDD
:103BFC00020E156F78EC09F09DEC0FF000C01FF36E
:103C0C0001C020F302C021F303C022F3730E0401A0
:103C1C00146F560E156F000E166F68EC05F01FC36F
:103C2C0001F420C302F421C303F422C304F4D50E1F
:103C3C000401056F020E066F020E076F3FEC0DF0CC
:103C4C00D50E146F020E156F78EC09F00B0E146F75
:103C5C00570E156F000E166F68EC05F00201D56B50
:103C6C00030129A949D0D50E04012E6F020E2F6F26
:103C7C00730E306F550E316F000E326FB3EC02F0D5
:103C8C001AC3FCF362EC0FF000C0FEF301C0FFF3AB
:103C9C00DB0E0301FC6F020EFD6F09EC0DF0D50E6F
:103CAC000401146F020E156F78EC09F00201D56B4C
:103CBC00D50E04012E6F020E2F6F640E306F550E51
:103CCC00316F000E326FB3EC02F019C3FCF362ECEF
:103CDC000FF000C0FEF301C0FFF3DB0E0301FC6F1D
:103CEC00020EFD6F09EC0DF0D50E0401146F020EDF
:103CFC00156F78EC09F009D00401900E146F550E75
:103D0C00156F000E166F68EC05F0F90E0401146FB8
:103D1C00560E156F000E166F68EC05F0000E83BE84
:103D2C00010E04012E6F300E2E273AEC05F0D00E4A
:103D3C000401146F560E156F000E166F68EC05F02B
:103D4C00000E87B6010E04012E6F300E2E273AECB2
:103D5C0005F0EC0E0401146F560E156F000E166F65
:103D6C0068EC05F0000E83B8010E04012E6F300EC6
:103D7C002E273AEC05F0E50E0401146F560E156F64
:103D8C00000E166F68EC05F0000E84B8010E0401ED
:103D9C002E6F300E2E273AEC05F04F0E0401146FE7
:103DAC00560E156F000E166F68EC05F0000E030131
:103DBC0029B5010E04012E6F300E2E273AEC05F0BA
:103DCC00D70E0401146F560E156F000E166F68ECAB
:103DDC0005F0000E030129BB010E04012E6F300EFD
:103DEC002E273AEC05F09C0E0401146F560E156F3D
:103DFC00000E166F68EC05F0000E80B0010E040189
:103E0C002E6F300E2E273AEC05F0DE0E0401146FE7
:103E1C00560E156F000E166F68EC05F0000E83BC85
:103E2C00010E04012E6F300E2E273AEC05F0EEEC4D
:103E3C0005F08EEC11F0030129BD2FD0245102089E
:103E4C0002E1235158081DE31FC304F020C305F001
:103E5C0021C306F022C307F0000E006E000E016EA7
:103E6C00580E026E830E036ECDEC07F0010ED8B027
:103E7C00000E006E005205E183AE03D087A601D080
:103E8C000BD0000E0201CF1902E1000ECE1904E195
:103E9C00030129A501D001D00DD1010E0201CE6F75
:103EAC00000ECF6F030129AB7ED08C9C2A0E256FA0
:103EBC00030E266F25C32EF426C32FF4460E0401E1
:103ECC00306F540E316F000E326FB3EC02F025C31D
:103EDC0014F426C315F478EC09F0EEEC05F0010EA1
:103EEC000401146F000E156F010E166F000E176F84
:103EFC0025C318F426C319F414EC06F05C0E0B6EF3
:103F0C00510E0C6E600E0D6E0D2EFED70C2EFCD7C6
:103F1C000B2EFAD70000770E146F4F0E156F000E94
:103F2C00166F68EC05F0F80E0301FC6F550EFD6F73
:103F3C00000EFE6F000E29B7010EFF6F7EEC0CF029
:103F4C007A0E0B6EC10E0C6E810E0D6E0D2EFED701
:103F5C000C2EFCD70B2EFAD700000000B30E040178
:103F6C00146F4D0E156F000E166F68EC05F0BA0E3F
:103F7C000301FC6F520EFD6F000EFE6F000E29B791
:103F8C00010EFF6F7EEC0CF01F0E0B6E710E0C6EA3
:103F9C001E0E0D6E0D2EFED70C2EFCD70B2EFAD747
:103FAC0000000301299B29AD51D029A94FD0C10E86
:103FBC000401146F4F0E156F000E166F68EC05F0B0
:103FCC00EEEC18F000C01AF300C0FCF325C3FDF3AF
:103FDC0026C3FEF340EC0CF025C314F426C315F4F1
:103FEC0078EC09F0EEEC05F02A0E0301256F030EB8
:103FFC00266F25C32EF426C32FF4240E0401306F34
:10400C00540E316F000E326FB3EC02F01AC3FCF396
:10401C0062EC0FF000C0FEF301C0FFF3070E0301CA
:10402C002525FC6F000E2621FD6F09EC0DF0020E0C
:10403C000401146F000E156F010E166F000E176F32
:10404C0025C318F426C319F414EC06F00401B80EB9
:10405C00146F530E156F000E166F68EC05F025C328
:10406C00BEF326C3BFF3EBEC13F000C0C6F201C0E5
:10407C00C7F200C014F401C015F4D50E166F020E71
:10408C00176F85EC05F0D50E146F020E156F78ECDA
:10409C0009F0EEEC05F025C3BEF326C3BFF357ECD5
:1040AC0012F0030129AD02D0299DF288A2EC09F08F
:1040BC00F8EC16F0000E2C1802E1010E2B18D8A407
:1040CC008BEF24F0030129BB8BEF24F0400E04018D
:1040DC00146F010E156F590E166F000E176FE7EC6B
:1040EC0006F000C040F201C041F2000E026E015019
:1040FC00025C02E100500008D8B089EF24F0010EF8
:10410C000401146F000E156F74EC06F0010E04011F
:10411C00146F000E156F010E166F000E176F350E13
:10412C00186F540E196F000E1A6FC2EC09F0490E7D
:10413C00146F4E0E156F000E166F68EC05F0280EFE
:10414C000401146F530E156F000E166FF7EC05F08B
:10415C00D60E0B6E110E0C6EE40E0D6E0D2EFED7E0
:10416C000C2EFCD70B2EFAD70000400E0401146F56
:10417C00010E156F78EC09F0EEEC05F00201746B92
:10418C00756B400E0401146F010E156F490E166FFE
:10419C00000E176FE7EC06F0000E026E0150025C89
:1041AC0002E10050000803E20201746B756B400ED3
:1041BC000401146F010E156F440E166F000E176F6D
:1041CC00E7EC06F0000E026E0150025C02E10050BA
:1041DC00000805E2010E0201746F000E756F400EAF
:1041EC000401146F010E156F4E0E166F000E176F33
:1041FC00E7EC06F000C040F201C041F2000E026E86
:10420C000150025C02E1005000087AE28A0E0401BF
:10421C002E6F020E2F6FAC0E306F500E316F000EE2
:10422C00326FB3EC02F0930E0401016F020E026FB9
:10423C00040E020140250401036F000E020141210E
:10424C000401046F0E0E056F000E066F42EC0AF0AF
:10425C00900E146F530E156F000E166F68EC05F070
:10426C00020E0401146F000E156F74EC06F0010EB3
:10427C000401146F000E156F010E166F000E176FF0
:10428C00130E186F540E196F000E1A6FC2EC09F052
:10429C00020E146F000E156F010E166F000E176FC5
:1042AC008A0E186F020E196F14EC06F08A0E146F3A
:1042BC00020E156F78EC09F0EEEC05F0A2EC09F0AB
:1042CC008A0E0301FC6F020EFD6F86EC0AF0B70E2E
:1042DC000B6EA10E0C6EC30E0D6E0D2EFED70C2E9A
:1042EC00FCD70B2EFAD700000000400E0401146F0F
:1042FC00010E156F78EC09F0EEEC05F0A2EC09F06C
:10430C00400E0401146F010E156F530E166F000E44
:10431C00176FE7EC06F000C040F201C041F2000E4E
:10432C00026E0150025C02E100500008D8B0E1D0EE
:10433C000201D56B100E0401146F560E156F000E92
:10434C00166F68EC05F0D50E0401016F020E026FBA
:10435C00050E020140250401036F000E02014121EC
:10436C000401046F080E056F000E066F42EC0AF094
:10437C00D50E146F020E156F78EC09F00201C66BA6
:10438C00C76B800ED36F000ED46FC86BC96B030163
:10439C00276B286B000E285D02E1080E275D2FE2CB
:1043AC00D50E2725E96E020E2821EA6EEE50300A52
:1043BC000AE0D50E2725E96E020E2821EA6EEE5092
:1043CC00310A01E003D00201C64BC72BD50E030105
:1043DC002725E96E020E2821EA6EEE50310A05E11E
:1043EC000201D351C827D451C9230201D433D3338A
:1043FC00D49FD4BDD48F0301274B282BCBD7000ED1
:10440C000201C71902E1080EC6195BE1030129A9D3
:10441C0058D0C8C219F3AC0E0401146F550E156FA9
:10442C00000E166F68EC05F019C3BEF344EC12F0E5
:10443C002A0E0301256F030E266F25C32EF426C307
:10444C002FF4E00E0401306F550E316F000E326FF9
:10445C00B3EC02F019C3FCF3D50E0301FD6F020E91
:10446C00FE6F40EC0CF025C3FCF326C3FDF3D50E18
:10447C000301FE6F020EFF6F32EC0FF025C32EF41A
:10448C0026C32FF4ECEC04F000C0C6F201C0C7F256
:10449C0000500301252504012E6F01500301262134
:1044AC0004012F6F610E306F560E316F000E326F9C
:1044BC00B3EC02F025C3BEF326C3BFF357EC12F0E6
:1044CC0016D0030129A90AD0780E0401146F4E0EE0
:1044DC00156F000E166F68EC05F009D0EB0E040199
:1044EC00146F500E156F000E166F68EC05F0A2ECF1
:1044FC0009F0400E0401146F010E156F6F0E166F4C
:10450C00000E176FE7EC06F000C040F201C041F25C
:10451C00000E026E0150025C02E1005000080DE238
:10452C0003012995FC0E0401146F520E156F000E39
:10453C00166F68EC05F0A2EC09F0400E0401146F44
:10454C00010E156F7A0E166F000E176FE7EC06F062
:10455C0000C040F201C041F2000E026E0150025C3C
:10456C0002E1005000080DE203012985F60E04015A
:10457C00146F510E156F000E166F68EC05F0A2EC5F
:10458C0009F0400E0401146F010E156F8C0E166F9E
:10459C00000E176FE7EC06F000C040F201C041F2CC
:1045AC00000E026E0150025C02E1005000081BE29A
:1045BC00DB0E0401146F510E156F000E166F68ECB4
:1045CC0005F025C3BEF326C3BFF3EBEC13F000C01C
:1045DC00C6F201C0C7F225C3BEF326C3BFF357EC26
:1045EC0012F0A2EC09F0400E0401146F010E156FCD
:1045FC00840E166F000E176FE7EC06F000C040F249
:10460C0001C041F2000E026E0150025C02E100504A
:10461C000008D8B0BFD0070E02014025E96E000E8D
:10462C004121EA6EEE50310A39E1080E40250401B1
:10463C00146F000E020141210401156F6B0E166FF1
:10464C00000E176FE7EC06F000C040F201C041F21B
:10465C00000E026E0150025C02E100500008D8A06E
:10466C008C88080E020140250401146F000E020113
:10467C0041210401156F5E0E166F000E176FE7ECEB
:10468C0006F000C040F201C041F2000E026E015073
:10469C00025C02E100500008D8A08C98070E0201C1
:1046AC004025E96E000E4121EA6EEE50320A39E1E6
:1046BC00080E40250401146F000E02014121040173
:1046CC00156F650E166F000E176FE7EC06F000C045
:1046DC0040F201C041F2000E026E0150025C02E198
:1046EC0000500008D8A08D88080E02014025040156
:1046FC00146F000E020141210401156F230E166F79
:10470C00000E176FE7EC06F000C040F201C041F25A
:10471C00000E026E0150025C02E100500008D8A0AD
:10472C008D98BF0E0401146F510E156F000E166F8D
:10473C0068EC05F025C32EF426C32FF45D0E04019E
:10474C00306F520E316F000E326FB3EC02F00E0E62
:10475C0003012525E16E000E2621E26E006A8CB85D
:10476C00002A300E002600C0E6FF150E2525E16E4E
:10477C00000E2621E26E006A8DB8002A300E00264B
:10478C0000C0E6FF25C3BEF326C3BFF357EC12F0FF
:10479C00A2EC09F0400E0401146F010E156F1B0EF4
:1047AC00166F000E176FE7EC06F000C040F201C068
:1047BC0041F2000E026E0150025C02E10050000852
:1047CC0041E2030129BB3ED0680E0401146F530E65
:1047DC00156F000E166F68EC05F025C32EF426C37A
:1047EC002FF43E0E0401306F530E316F000E326FFA
:1047FC00B3EC02F025C3BEF326C3BFF357EC12F0A3
:10480C004C0E0401146F500E156F000E166F68ECF1
:10481C0005F0EC0E0301FC6F550EFD6F000EFE6FE4
:10482C00000E29B7010EFF6F7EEC0CF0AC0E0401EC
:10483C00146F560E156F000E166F68EC05F08C8C0D
:10484C000301298B400E0401146F010E156FA40E89
:10485C00166F000E176FE7EC06F000C040F201C0B7
:10486C0041F2000E026E0150025C02E100500008A1
:10487C0023E2EF0E0401146F530E156F000E166F2A
:10488C0068EC05F02A0E0301256F030E266F25C375
:10489C002EF426C32FF4D20E0401306F4B0E316F61
:1048AC00000E326FB3EC02F025C3BEF326C3BFF388
:1048BC0057EC12F0A2EC09F0030129BB24D0E60E50
:1048CC000401146F4D0E156F000E166F68EC05F099
:1048DC00E60E0301FC6F520EFD6F000EFE6F000E14
:1048EC0029B7010EFF6F7EEC0CF00D0E0B6E2D0E2A
:1048FC000C6ED70E0D6E0D2EFED70C2EFCD70B2E7C
:10490C00FAD700000000A2EC09F00201724B732BE5
:10491C00800E006E800E7319005C02E172513B0830
:10492C0004E2CE6BCF6B726B736B000E2E1802E130
:10493C00010E2D18D8A498D0340E0401146F550E06
:10494C00156F000E166F68EC05F0BC0E0401146FA9
:10495C00000E156F78EC09F0EEEC05F0BC0E0401BE
:10496C002E6F000E2F6F9E0E306F000E316F050EE6
:10497C00326F09EC05F0000E011802E1000E001870
:10498C0005E1010E0201D06F000ED16FBC0E0401C7
:10499C002E6F000E2F6FA90E306F000E316F060EAA
:1049AC00326F09EC05F0000E011802E1000E001840
:1049BC0003E10201D06BD16BBC0E04012E6F000E13
:1049CC002F6FB00E306F000E316F050E326F09EC89
:1049DC0005F0000E011802E1000E0018D8B48C8C02
:1049EC00BC0E04012E6F000E2F6FB60E306F000E32
:1049FC00316F050E326F09EC05F0000E011802E163
:104A0C00000E0018D8B48C9C030129AB20D0BC0E2E
:104A1C00FC6F000EFD6F86EC0AF00D0E04012E6F7C
:104A2C0061EC05F0990E0B6E310E0C6EA20E0D6E34
:104A3C000D2EFED70C2EFCD70B2EFAD70000400EF5
:104A4C000401146F010E156F78EC09F009D0040104
:104A5C002C0E146F500E156F000E166F68EC05F0CF
:104A6C00A2EC09F0F8EC16F0000E2C1802E1020E84
:104A7C002B181EE1860E0401146F510E156F000EDB
:104A8C00166F68EC05F063C014F464C015F4D50E11
:104A9C000401166F020E176F85EC05F0D50E146F1E
:104AAC00020E156F78EC09F0EEEC05F0A2EC09F0B3
:104ABC00000E2E1802E1020E2D1824E118C0C6F2C9
:104ACC0019C0C7F2F8EC16F08C0E0401146F500EDE
:104ADC00156F000E166F68EC05F0C6C214F4C7C251
:104AEC0015F4D50E0401166F020E176F85EC05F048
:104AFC00D50E146F020E156F78EC09F0EEEC05F084
:104B0C00F8EC16F080B002D0030129950301000ED9
:104B1C00AB1902E1000EAA1901E1F8D795EF1DF0CF
:024B2C00FFD7B1
:1057140010EE18F0A40E006E010E016E2E0EF66E41
:0E5724004B0EF76E000EF86EBDEC10F012008A
:024B2E00000085
:014B30000084
:084B3100536F6D6D65696C00A6
:054B3900204F6666003C
:034B3E004F4B00DA
:024B4100000072
:024B4300000070
:024B450000006E
:064B47004572726F72005E
:034B4D004F4B00CB
:074B50002B43474D533A00CF
:034B57004F4B00C1
:054B5A00333833370081
:054B5F00343731350080
:054B64004D41483D0039
:064B69004D4350313D00F8
:054B6F00434D54490014
:054B7400204F66660001
:024B790000003A
:044B7B00204F6E0059
:024B7F00000034
:044B8100204F6E0053
:0B4B8500537572766579204F6666005C
:0A4B9000537572766579204F6E00B0
:084B9A00436465204C656400D2
:0F4BA20044617461204F6E2044656D616E640044
:014BB100748F
:024BB200000001
:064BB40044656275670014
:054BBA0048656C70006D
:074BBF004E6F726D616C0086
:064BC6004454523D310091
:064BCC004454523D30008C
:104BD2000D0A4364657320646973706F3A0D0A208D
:104BE20044617461204F6E2064656D616E64200DB6
:104BF2000A20537572766579204F6E20286F7520D2
:104C02004F6666290D0A20536F6D6D65696C0D0A3A
:104C120020436465204C65643120306E20286F7516
:104C2200204F6666290D0A204D41483D31352F300F
:104C3200392F32392C31363A34353A30302B303440
:104C42000D0A204D4350313D30303030303030305D
:034C52000D0A0048
:104C55002031384638374A35305F47534D325F5536
:104C6500415254325F55415254315F4C43445F4980
:104C750032435F4D435032333031375F57616B6597
:104C850055705F4F6E4576656E745F313531315FB6
:104C9500775F682E6D637070692056657273696FF2
:104CA5006E203A2030332D30322D323031360D0A18
:014CB50000FE
:104CB6002031384638374A35305F47534D325F55D5
:104CC600415254325F55415254315F4C43445F491F
:104CD60032435F4D435032333031375F57616B6536
:104CE60055705F4F6E4576656E745F313630323083
:0A4CF600335F775F682E630D0A003C
:104D0000205665726966696572206C61207072E96F
:104D100073656E6365206465207265736973746181
:104D20006E6365732050756C6C20555020737572DE
:0F4D30002053434C20657420534441200D0A004A
:104D3F0020496E69742056425241592055415254B0
:104D4F00312031393230302C382C4E2C31206574D3
:104D5F00205155454354454C205541525432203132
:0D4D6F00393230302C382C4E2C310D0A001A
:104D7C00204C69737420616C6C20554E5245414433
:104D8C00206D73672066726F6D20696E626F78207C
:104D9C002841542B434D474C3D52454320554E52D0
:074DAC00454144290D0A00F6
:104DB30045666661636520746F7573206C65732047
:104DC300534D53207265E77573202841542B514D81
:104DD3004744413D2244454C20494E424F582229E5
:034DE3000D0A00B6
:104DE60045666661636520746F7573206C65732014
:104DF600534D53207265E77573202841542B514D4E
:104E06004744413D2244454C20494E424F582229B1
:034E16000D0A0082
:104E1900205465737420736920656E7265676973C0
:104E29007472E920737572206C652072657365610F
:104E390075202841542B435245473F31290D0A001B
:104E49002052656164206D657373616765204E4FFB
:104E59004E204C5553202841542B434D474C3D225D
:0F4E690052454320554E5245414422290D0A001F
:104E7800205265667573E965200D0A20504220644A
:104E88006520666F726D617420636465203A204DF9
:0F4E98004350313D30303030303030300D0A0073
:104EA700222B333336323133333437313522002234
:104EB7002B333336313431333338333722004E6FA7
:0D4EC7007420617574686F72697A6564000B
:104ED40020466169726520526573657420706F7530
:104EE400722072656C616E636572206C65207072ED
:0B4EF4006F6772616D652E2E0D0A00C5
:104EFF0020557361676520646520534C45455020EC
:104F0F006D6F646520302065742032202C20204383
:0A4F1F00646520445452200D0A007E
:104F2900204E6576657220676F20696E20534C4567
:104F39004550206D6F64652841542B5153434C4BA8
:074F49003D3029200D0A0094
:104F5000204C6563747572652064652064617465B6
:104F6000206574206865757265202841542B434381
:074F70004C4B3F290D0A0024
:104F77004E6576657220476F20696E20534C454514
:104F870050206D6F64652841542B5153434C4B3D62
:064F97003029200D0A0084
:104F9D002031657265204C656374757265204144DE
:104FAD004320524131206574204144432052413207
:044FBD00200D0A00B9
:104FC10057616B65557020766961206368616E6712
:104FD10065206F6E203845204D43503233303137D4
:044FE100203A200052
:104FE5002031657265204C65637475726520414496
:104FF50043205241312065742041444320524132BF
:04500500200D0A0070
:10500900200D0A436F6E737469747574696F6E202D
:10501900647520534D5320E020656E766F79657273
:035029000D0A006D
:10502C00200D0A2070726F626C656D6F2047534DB6
:10503C003220656E20736F6D6D65696C200D0A00F2
:10504C00476F20696E20534C454550206D6F646549
:10505C002841542B5153434C4B3D3229200D0A000F
:10506C0020506F776572204F4E206D6F64756C65A4
:10507C002047534D322D636C69636B200D0A200061
:10508C000D0A204465626F7264656D656E74204212
:10509C00756666657231205541525431203A2000B4
:1050AC0041542B43434C4B3D2231352F30392F3259
:1050BC00392C31363A34353A30302B3034220D001D
:1050CC000D0A496E6974206574203165722044653F
:0F50DC006D6172726167652047534D320D0A0096
:1050EB00205265667573E96520636172204D4350EC
:0F50FB00323330313720616273656E740D0A00F5
:10510A002031393230302042617564207261746511
:0F511A00204E65676F636520424144200D0A00F7
:1051290020496E6974204D4350323330313720386D
:0F5139004520385320656E20493243200D0A006F
:10514800205365742050494E20636F64652841548C
:0F5158002B4350494E3D3132333429200D0A008C
:10516700200D0A20436F6E74656E75206475205399
:0F5177004D5320E020656E766F7965720D0A004A
:10518600204465626F7264656D656E742062756633
:0D519600666572205541525432200D0A000A
:1051A300205072657420706F757220656E766F691A
:0C51B300204D736720747874200D0A00F2
:1051BF00205265746F75722064276F726472652058
:0C51CF00636465204C656473200D0A00C9
:1051DB000D0A456E766F69204461746173206465B6
:0B51EB006D616E64E96573200D0A0021
:1051F600204469616C6F67756520534D5320726555
:0A5206007461626C6974200D0A00E7
:1052100020546573742070726573656E6365204CED
:0A522000434420323131390D0A00F9
:10522A0020436F6D706F7365204E756D65726F20C8
:0A523A002841542B434D47533D001B
:10524400204572726575722073757220656E766F73
:095254006920534D53200D0A009E
:10525D000D0A5265746F7572204C6564313D2020C6
:08526D004C6564323D200D0088
:10527500204E622064652070617320496E69742038
:075285004C4344203D2000D2
:10528C002041726D6520525820495420554152548A
:07529C0031202E2E0D0A0047
:1052A3002041726D65205258204954205541525473
:0752B30032202E2E0D0A002F
:1052BA0041542B514D4744413D2244454C20494ECF
:0652CA00424F58220D00C6
:1052D0000D0A47534D322050494331384638374A3A
:0652E00035303A0D0A0012
:1052E60041542B514D4744413D2244454C20494EA3
:0652F600424F58220D009A
:1052FC002053544F50206469616C6F67756520535F
:06530C004D53200D0A00C4
:1053120041542B434D474C3D2252454320554E525A
:06532200454144220D008C
:1053280041542B434D474C3D2252454320554E5244
:06533800454144220D0076
:10533E000D0A4F4B206D6F6465206D696D696E753A
:05534E006D20780D0048
:10535300204E65676F6365206261756420726174B6
:0553630065200D0A00A9
:10536800204D69736520656E20736F6D6D65696C7E
:04537800200D0A00FA
:10537C0020496E69742049324331203130304B68FA
:04538C007A0D0A008C
:10539000204D414A2064617465206574204865751C
:0453A0007265200012
:1053A40020496E697420446973706C6179204C43A0
:0453B400440D0A009A
:1053B80020436F6D706F7365204D7367206C656E49
:0353C8003D200085
:1053CB00204E65676F636520726575737369200D79
:0253DB000A00C6
:1053DD00205068617365206427696E697420656E5D
:0253ED0020009E
:1053EF002048656C702064656D616E64E965200D01
:0253FF000A00A2
:10540100204572723A204E6F204D43503233303175
:02541100370062
:105413004D414A206461746520686575726520207A
:015423000088
:105424003820496E703D202020202020202020207C
:015434000077
:10543500526563657074696F6E20534D532020204B
:015445000066
:1054460052657665696C2047534D32202F4454527D
:015456000055
:1054570020526573657420436C69636B65723220F3
:015467000044
:1054680020496E74727573696F6E204541313D2015
:015478000033
:1054790053543D20202044493D2020534F3D2020B6
:015489000022
:10548A0053746570203A202E2E2E2E2E2F20352072
:01549A000011
:10549B00202020202020706173202F2035202020F9
:0154AB000000
:1054AC004E65676F63652062617564207261746517
:0154BC0000EF
:1054BD00436F6D706F7365204E756D65726F202033
:0154CD0000DE
:1054CE005068617365206427696E697420656E206B
:0154DE0000CD
:1054DF00496E69742047534D322D436C69636B20BD
:0154EF0000BC
:1054F00041647265737365204F4B203078343020DF
:0155000000AA
:10550100696E69204D43503233303137204932437F
:015511000099
:1055120042414420416472657373203078343020F4
:015522000088
:1055230042414420496E69742053746570202020E1
:015533000077
:1055340020526563657074205541525431203A00FD
:10554400436865636B204465766963652040200089
:1055540020456E766F6920534D53204F4B203A00FF
:0F5564003B2038533D2030303030303030300075
:0F5573003B2038453D2030303030303030300074
:0E55820041542B4350494E3D313233340D001D
:0E5590003B204E6F204D4350323330313700F8
:0E559E00206973206E6F7420666F756E640056
:0D55AC0020416363657074E965200D0A00FD
:0D55B90038533D203030303030303030007D
:0D55C6002041444320496E6974200D0A0005
:0D55D30038453D2030303030303030300071
:0C55E00020436465204D435031203D0005
:0C55EC0041542B5153434C4B3D320D00F9
:0C55F80041542B5153434C4B3D300D00EF
:0C56040041542B5153434C4B3D300D00E2
:0C561000436465204D435031203A2000D7
:0B561C003B20454132204E6F773D00DF
:0A5627000D0A20456E642E0D0A00E6
:0A56310020666F756E64204F4B0079
:0A563B0041542B43434C4B3F0D003C
:0A56450041542B435245473F0D002E
:09564F003B4469616C6F673D008A
:0956580020464F5343203D200081
:09566100202E2E4F4B200D0A00F3
:09566A0041542B434D47533D0010
:095673003B54656D70463D2000BA
:08567C0020425032203D2000C5
:0856840020425031203D2000BE
:08568C00204C4431203D2000B8
:085694002054656D703D2000FB
:08569C003B20535441543D0032
:0856A400204C4432203D20009F
:0856AC004454523D310D0A0087
:0756B400207061732F350027
:0756BB0054656D703D2000F5
:0756C20020537465703A00EB
:0756C9002E2E424144210096
:0756D0003B204250323D0077
:0756D7003B20534F4D3D0045
:0756DE003B204454523D0043
:0756E5003B204C44323D0064
:0756EC003B204C44313D005E
:0656F3004541313D20009D
:0656F9003B4250313D0070
:0656FF00204541313D0091
:065705002E2E204F4B0088
:05570B00646567200049
:0457100041540D00F3
:020000040001F9
:06FFF800ACF705FFF0FF6D
:00000001FF
